:100000000C9434000C9446000C9446000C9446006A
:100010000C9446000C9446000C9446000C94460048
:100020000C9446000C9446000C9446000C94460038
:100030000C9446000C9446000C9446000C94460028
:100040000C9446000C9446000C9446000C94460018
:100050000C9446000C9446000C9446000C94460008
:100060000C9446000C94460011241FBECFEFD8E03C
:10007000DEBFCDBF21E0A0E0B1E001C01D92A23003
:10008000B207E1F70E9491000C949F000C940000CD
:10009000389A90E031E09817D1F028B1232728B999
:1000A0002FEF4FE756E1215040405040E1F700C0AC
:1000B000000028B1232728B92FEF4FE756E1215040
:1000C00040405040E1F700C000009F5FE4CF08953A
:1000D00087B1897F87B988B1897F88B9089586B14A
:1000E000867090E09595879520910101281749F039
:1000F0008093010190910001990F990F892B8093B2
:100100000001809100018B3431F0873841F4109266
:10011000000182E008951092000181E0089580E0DE
:1001200008950E94680082E00E9448000E946F00CB
:10013000813019F08230B9F3F9CF81E0F5CFF8942E
:02014000FFCFEF
:00000001FF
